 touch

 Timestamp is 4fb05c6d (Mon May 14 13:14:21 2012)

 Preferred load address is 10000000

 Start         Length     Name                   Class
 0001:00000000 00000d3eH .rdata                  CODE
 0001:00000d40 00000022H .rdata$debug            CODE
 0001:00000d64 00004b60H .text                   CODE
 0001:000058c4 00000018H .xdata                  CODE
 0001:000058dc 00000014H .idata$2                CODE
 0001:000058f0 00000014H .idata$3                CODE
 0001:00005904 00000084H .idata$4                CODE
 0001:00005988 0000000cH .idata$6                CODE
 0001:000059a0 00000161H .edata                  CODE
 0002:00000000 00000084H .idata$5                DATA
 0002:00000088 00000538H .data                   DATA
 0002:000005c0 0000016cH .bss                    DATA
 0003:00000000 00000190H .pdata                  DATA

  Address         Publics by Value              Rva+Base       Lib:Object

 0000:00000000       ___safe_se_handler_table   00000000     <absolute>
 0000:00000000       ___safe_se_handler_count   00000000     <absolute>
 0001:0000001c       MIN_CAL_COUNT              1000101c     touch.obj
 0001:00000020       ??_C@_1M@EPBPGMBG@?$AAA?$AAD?$AAC?$AA1?$AA?3?$AA?$AA@ 10001020     touch.obj
 0001:00000030       ??_C@_1GE@MOAFGNMM@?$AAE?$AAR?$AAR?$AAO?$AAR?$AA?3?$AA?5?$AAF?$AAa?$AAi?$AAl?$AAe?$AAd?$AA?5?$AAt?$AAo?$AA?5?$AAr?$AAe?$AAq?$AAu?$AAe?$AAs?$AAt?$AA?5?$AAt?$AAh?$AAe?$AA?5?$AAg?$AAI?$AAn@ 10001030     touch.obj
 0001:00000094       ??_C@_1CK@OFGGHANN@?$AA?$CL?$AAT?$AAo?$AAu?$AAc?$AAh?$AA?5?$AAs?$AAc?$AAr?$AAe?$AAe?$AAn?$AA?5?$AAI?$AAn?$AAi?$AAt?$AA?$AN?$AA?6?$AA?$AA@ 10001094     touch.obj
 0001:000000c0       ??_C@_1GE@DHLKOKNH@?$AAE?$AAR?$AAR?$AAO?$AAR?$AA?3?$AA?5?$AAF?$AAa?$AAi?$AAl?$AAe?$AAd?$AA?5?$AAt?$AAo?$AA?5?$AAr?$AAe?$AAl?$AAe?$AAa?$AAs?$AAe?$AA?5?$AAt?$AAh?$AAe?$AA?5?$AAg?$AAI?$AAn@ 100010c0     touch.obj
 0001:00000124       ??_C@_1CI@OHCJFJPM@?$AAE?$AAR?$AAR?$AAO?$AAR?$AA?3?$AA?5?$AA?$CF?$AAs?$AA?5?$AAl?$AAi?$AAn?$AAe?$AA?5?$AA?$CF?$AAd?$AA?3?$AA?5?$AA?$AA@ 10001124     touch.obj
 0001:00000150       ??_C@_1JE@MHINAMCB@?$AAC?$AA?3?$AA?2?$AAW?$AAI?$AAN?$AAC?$AAE?$AAR?$AAO?$AAO?$AAT?$AAS?$AA?2?$AAT?$AAo?$AAp?$AAa?$AAz?$AA?2?$AAW?$AAI?$AAN?$AAC?$AAE?$AA6?$AA0?$AA0?$AA?2?$AAP?$AAL?$AAA@ 10001150     touch.obj
 0001:000001e8       ??_C@_1FM@GOBOJOFI@?$AAT?$AAo?$AAu?$AAc?$AAh?$AAP?$AAa?$AAn?$AAe?$AAl?$AAG?$AAe?$AAt?$AAD?$AAe?$AAv?$AAi?$AAc?$AAe?$AAC?$AAa?$AAp?$AAs?$AA?3?$AA?5?$AAi?$AAn?$AAv?$AAa?$AAl?$AAi?$AAd@ 100011e8     touch.obj
 0001:00000248       ??_C@_1FK@FNONLNGN@?$AA?$CF?$AAs?$AA?3?$AA?5?$AAD?$AAE?$AAB?$AAU?$AAG?$AAC?$AAH?$AAK?$AA?5?$AAf?$AAa?$AAi?$AAl?$AAe?$AAd?$AA?5?$AAi?$AAn?$AA?5?$AAf?$AAi?$AAl?$AAe?$AA?5?$AA?$CF?$AAs?$AA?5?$AAa@ 10001248     touch.obj
 0001:000002a8       ??_C@_1FI@DOMOKNDA@?$AAD?$AAd?$AAs?$AAi?$AAT?$AAo?$AAu?$AAc?$AAh?$AAP?$AAa?$AAn?$AAe?$AAl?$AAS?$AAe?$AAt?$AAM?$AAo?$AAd?$AAe?$AA?5?$AA?3?$AA?5?$AAU?$AAn?$AAs?$AAu?$AAp?$AAp?$AAo?$AAr@ 100012a8     touch.obj
 0001:00000300       ??_C@_1GC@IBMOGKMF@?$AAD?$AAd?$AAs?$AAi?$AAT?$AAo?$AAu?$AAc?$AAh?$AAP?$AAa?$AAn?$AAe?$AAl?$AAS?$AAe?$AAt?$AAM?$AAo?$AAd?$AAe?$AA?5?$AA?3?$AA?5?$AAS?$AAe?$AAt?$AA?5?$AAS?$AAa?$AAm?$AAp@ 10001300     touch.obj
 0001:00000368       ??_C@_1GE@KNOEACMA@?$AAD?$AAd?$AAs?$AAi?$AAT?$AAo?$AAu?$AAc?$AAh?$AAP?$AAa?$AAn?$AAe?$AAl?$AAS?$AAe?$AAt?$AAM?$AAo?$AAd?$AAe?$AA?5?$AA?3?$AA?5?$AAS?$AAe?$AAt?$AA?5?$AAS?$AAa?$AAm?$AAp@ 10001368     touch.obj
 0001:000003cc       ??_C@_1CO@IBMILJAB@?$AA?7?$AAC?$AAa?$AAl?$AAi?$AAb?$AAr?$AAa?$AAt?$AAi?$AAo?$AAn?$AA?5?$AAf?$AAa?$AAi?$AAl?$AAe?$AAd?$AA?4?$AA?$AN?$AA?6?$AA?$AA@ 100013cc     tch_cal:calibrat.obj
 0001:00000400       ??_C@_1FO@JLBFGOAH@?$AAT?$AAo?$AAu?$AAc?$AAh?$AAP?$AAa?$AAn?$AAe?$AAl?$AAS?$AAe?$AAt?$AAC?$AAa?$AAl?$AAi?$AAb?$AAr?$AAa?$AAt?$AAi?$AAo?$AAn?$AA?3?$AA?5?$AAd?$AAe?$AAl?$AAt?$AAa?$AA?5@ 10001400     tch_cal:calibrat.obj
 0001:00000460       ??_C@_1DG@BBHLEELA@?$AAc?$AAa?$AAl?$AAi?$AAb?$AAr?$AAa?$AAt?$AAi?$AAn?$AAg?$AA?5?$AA?$CF?$AAd?$AA?5?$AAp?$AAo?$AAi?$AAn?$AAt?$AA?5?$AAs?$AAe?$AAt?$AA?$AN?$AA?6?$AA?$AA@ 10001460     tch_cal:calibrat.obj
 0001:00000498       ??_C@_1GI@MGLMFFFE@?$AAM?$AAa?$AAx?$AAi?$AAm?$AAu?$AAm?$AA?5?$AAe?$AAr?$AAr?$AAo?$AAr?$AA?5?$AA?$CF?$AAu?$AA?5?$AAe?$AAx?$AAc?$AAe?$AAe?$AAd?$AAs?$AA?5?$AAc?$AAa?$AAl?$AAi?$AAb?$AAr?$AAa@ 10001498     tch_cal:calibrat.obj
 0001:00000500       ??_C@_1II@DJLOMFPA@?$AAM?$AAa?$AAx?$AAi?$AAm?$AAu?$AAm?$AA?5?$AAe?$AAr?$AAr?$AAo?$AAr?$AA?5?$AA?$CI?$AAs?$AAq?$AAu?$AAa?$AAr?$AAe?$AA?5?$AAo?$AAf?$AA?5?$AAE?$AAu?$AAc?$AAl?$AAi?$AAd?$AAe@ 10001500     tch_cal:calibrat.obj
 0001:00000588       ??_C@_1DG@NEEPBIEH@?$AA?$CI?$AA?$CF?$AA4?$AAd?$AA?0?$AA?5?$AA?$CF?$AA4?$AAd?$AA?$CJ?$AA?5?$AA?$DN?$AA?$DO?$AA?5?$AA?$CI?$AA?$CF?$AA4?$AAd?$AA?0?$AA?5?$AA?$CF?$AA4?$AAd?$AA?$CJ?$AA?$AN?$AA?6?$AA?$AA@ 10001588     tch_cal:calibrat.obj
 0001:000005c0       ??_C@_1DI@KOEAOJB@?$AA?5?$AA?5?$AA?5?$AAS?$AAc?$AAr?$AAe?$AAe?$AAn?$AA?5?$AA?5?$AA?5?$AA?5?$AA?$DN?$AA?$DO?$AA?5?$AA?5?$AA?5?$AA?5?$AAM?$AAa?$AAp?$AAp?$AAe?$AAd?$AA?$AN?$AA?6?$AA?$AA@ 100015c0     tch_cal:calibrat.obj
 0001:000005f8       ??_C@_1CO@HGFEBAFC@?$AAC?$AAa?$AAl?$AAi?$AAb?$AAr?$AAa?$AAt?$AAi?$AAo?$AAn?$AA?5?$AAR?$AAe?$AAs?$AAu?$AAl?$AAt?$AAs?$AA?3?$AA?$AN?$AA?6?$AA?$AA@ 100015f8     tch_cal:calibrat.obj
 0001:00000628       ??_C@_1DI@HBBBNELP@?$AAM?$AAa?$AAx?$AAi?$AAm?$AAu?$AAm?$AA?5?$AAA?$AAl?$AAl?$AAo?$AAw?$AAe?$AAd?$AA?5?$AAE?$AAr?$AAr?$AAo?$AAr?$AA?5?$AA?$CF?$AAd?$AA?3?$AA?$AN?$AA?6?$AA?$AA@ 10001628     tch_cal:calibrat.obj
 0001:00000660       ??_C@_1BI@KKLLCJMC@?$AAM?$AAa?$AAx?$AAC?$AAa?$AAl?$AAE?$AAr?$AAr?$AAo?$AAr?$AA?$AA@ 10001660     tch_cal:calibrat.obj
 0001:00000678       ??_C@_1DC@PPKDPGKC@?$AAH?$AAA?$AAR?$AAD?$AAW?$AAA?$AAR?$AAE?$AA?2?$AAD?$AAE?$AAV?$AAI?$AAC?$AAE?$AAM?$AAA?$AAP?$AA?2?$AAT?$AAO?$AAU?$AAC?$AAH?$AA?$AA@ 10001678     tch_cal:calibrat.obj
 0001:000006ac       ??_C@_1BA@LEPJIIOK@?$AAU?$AAn?$AAk?$AAn?$AAo?$AAw?$AAn?$AA?$AA@ 100016ac     tch_cal:largenum.obj
 0001:000006c0       ??_C@_1HA@ENPKAGOE@?$AAC?$AA?3?$AA?2?$AAy?$AAm?$AAz?$AAk?$AAi?$AA?2?$AAp?$AAu?$AAb?$AAl?$AAi?$AAc?$AA?2?$AAC?$AAO?$AAM?$AAM?$AAO?$AAN?$AA?2?$AAo?$AAa?$AAk?$AA?2?$AAd?$AAr?$AAi?$AAv?$AAe@ 100016c0     tch_cal:largenum.obj
 0001:00000730       ??_C@_1HI@KLEMONDH@?$AAC?$AA?3?$AA?2?$AAy?$AAm?$AAz?$AAk?$AAi?$AA?2?$AAp?$AAu?$AAb?$AAl?$AAi?$AAc?$AA?2?$AAC?$AAO?$AAM?$AAM?$AAO?$AAN?$AA?2?$AAo?$AAa?$AAk?$AA?2?$AAd?$AAr?$AAi?$AAv?$AAe@ 10001730     tchmdd:tchbasic.obj
 0001:000007a8       ??_C@_1CK@KALIMGPI@?$AAD?$AAl?$AAl?$AA?5?$AAP?$AAr?$AAo?$AAc?$AAe?$AAs?$AAs?$AA?5?$AAD?$AAe?$AAt?$AAa?$AAc?$AAh?$AA?$AN?$AA?6?$AA?$AA@ 100017a8     tchmdd:tchbasic.obj
 0001:000007d4       ??_C@_1DG@ODCFLDLG@?$AAD?$AAd?$AAs?$AAi?$AAT?$AAo?$AAu?$AAc?$AAh?$AAP?$AAa?$AAn?$AAe?$AAl?$AAA?$AAt?$AAt?$AAa?$AAc?$AAh?$AA?5?$AA?$DO?$AA?5?$AA1?$AA?$AN?$AA?6?$AA?$AA@ 100017d4     tchmdd:tchbasic.obj
 0001:0000080c       ??_C@_1CK@MANAIBA@?$AAD?$AAl?$AAl?$AA?5?$AAP?$AAr?$AAo?$AAc?$AAe?$AAs?$AAs?$AA?5?$AAA?$AAt?$AAt?$AAa?$AAc?$AAh?$AA?$AN?$AA?6?$AA?$AA@ 1000180c     tchmdd:tchbasic.obj
 0001:00000838       ??_C@_1II@DGCOIMLP@?$AAT?$AAo?$AAu?$AAc?$AAh?$AAP?$AAa?$AAn?$AAe?$AAl?$AAE?$AAn?$AAa?$AAb?$AAl?$AAe?$AA?3?$AA?5?$AAI?$AAn?$AAt?$AAe?$AAr?$AAr?$AAu?$AAp?$AAt?$AAI?$AAn?$AAi?$AAt?$AAi@ 10001838     tchmdd:tchmain.obj
 0001:000008c0       ??_C@_1HK@PKLFBBPC@?$AAT?$AAo?$AAu?$AAc?$AAh?$AAP?$AAa?$AAn?$AAe?$AAl?$AAE?$AAn?$AAa?$AAb?$AAl?$AAe?$AA?3?$AA?5?$AAI?$AAn?$AAt?$AAe?$AAr?$AAr?$AAu?$AAp?$AAt?$AAI?$AAn?$AAi?$AAt?$AAi@ 100018c0     tchmdd:tchmain.obj
 0001:0000093c       ??_C@_1DC@GDGJFAPL@?$AA?$CF?$AAd?$AA?5?$AAd?$AAo?$AAw?$AAn?$AA?5?$AAs?$AAa?$AAm?$AAp?$AAl?$AAe?$AAs?$AA?5?$AAq?$AAu?$AAe?$AAu?$AAe?$AAd?$AA?$AN?$AA?6?$AA?$AA@ 1000193c     tchmdd:tchmain.obj
 0001:00000970       ??_C@_1FK@PCOIIHBJ@?$AA?$CK?$AA?$CK?$AA?$CK?$AA?$CK?$AA?5?$AAQ?$AAu?$AAe?$AAu?$AAi?$AAn?$AAg?$AA?5?$AAp?$AAo?$AAi?$AAn?$AAt?$AA?5?$AA?$CI?$AA?$CF?$AAd?$AA?0?$AA?5?$AA?$CF?$AAd?$AA?$CJ?$AA?0?$AA?5?$AAf?$AAl?$AAa@ 10001970     tchmdd:tchmain.obj
 0001:000009cc       ??_C@_1DI@KAFCCODB@?$AAM?$AA?5?$AA?$CF?$AAl?$AAd?$AA?0?$AA?$CF?$AAl?$AAd?$AA?5?$AA?5?$AA?$CF?$AAl?$AAd?$AA?0?$AA?$CF?$AAl?$AAd?$AA?5?$AA?5?$AA?$CF?$AAl?$AAd?$AA?0?$AA?$CF?$AAl?$AAd?$AA?$AA@ 100019cc     tchmdd:tchmain.obj
 0001:00000a08       ??_C@_1GC@FJOPAGMC@?$AA?$CK?$AA?$CK?$AA?$CK?$AA?$CK?$AA?5?$AAC?$AAa?$AAl?$AAi?$AAb?$AAr?$AAa?$AAt?$AAi?$AAo?$AAn?$AA?5?$AAp?$AAo?$AAi?$AAn?$AAt?$AA?5?$AA?$CI?$AA?$CF?$AAd?$AA?0?$AA?5?$AA?$CF?$AAd?$AA?$CJ?$AA?0@ 10001a08     tchmdd:tchmain.obj
 0001:00000a6c       ??_C@_1BG@FLJCGFBL@?$AAT?$AAC?$AAH?$AA_?$AAI?$AAN?$AAT?$AAR?$AA?$AN?$AA?6?$AA?$AA@ 10001a6c     tchmdd:tchmain.obj
 0001:00000a88       ??_C@_1FA@JCKIIMMD@?$AAT?$AAO?$AAU?$AAC?$AAH?$AA?3?$AAT?$AAh?$AAr?$AAd?$AAP?$AAr?$AAi?$AAo?$AA?5?$AA?$DN?$AA?5?$AA?$CF?$AAd?$AA?0?$AA?5?$AAT?$AAh?$AAr?$AAd?$AAH?$AAi?$AAg?$AAh?$AAP?$AAr?$AAi@ 10001a88     tchmdd:tchmain.obj
 0001:00000ad8       ??_C@_1CA@IHOLOKEO@?$AAH?$AAi?$AAg?$AAh?$AAP?$AAr?$AAi?$AAo?$AAr?$AAi?$AAt?$AAy?$AA2?$AA5?$AA6?$AA?$AA@ 10001ad8     tchmdd:tchmain.obj
 0001:00000af8       ??_C@_1JE@CEGKFACG@?$AAT?$AAO?$AAU?$AAC?$AAH?$AA?3?$AAT?$AAo?$AAu?$AAc?$AAh?$AAP?$AAa?$AAn?$AAe?$AAl?$AAp?$AAG?$AAe?$AAt?$AAP?$AAr?$AAi?$AAo?$AAr?$AAi?$AAt?$AAy?$AA?5?$AA?9?$AA?5?$AAF@ 10001af8     tchmdd:tchmain.obj
 0001:00000b8c       ??_C@_1BI@BHLBGEOK@?$AAP?$AAr?$AAi?$AAo?$AAr?$AAi?$AAt?$AAy?$AA2?$AA5?$AA6?$AA?$AA@ 10001b8c     tchmdd:tchmain.obj
 0001:00000ba8       ??_C@_1LI@IHCCBOIO@?$AAT?$AAO?$AAU?$AAC?$AAH?$AA?3?$AAT?$AAo?$AAu?$AAc?$AAh?$AAP?$AAa?$AAn?$AAe?$AAl?$AAp?$AAG?$AAe?$AAt?$AAP?$AAr?$AAi?$AAo?$AAr?$AAi?$AAt?$AAy?$AA?5?$AA?9?$AA?5?$AAR@ 10001ba8     tchmdd:tchmain.obj
 0001:00000c60       ??_C@_1CO@HCHNLANK@?$AA?2?$AAD?$AAr?$AAi?$AAv?$AAe?$AAr?$AAs?$AA?2?$AAB?$AAu?$AAi?$AAl?$AAt?$AAI?$AAn?$AA?2?$AAT?$AAo?$AAu?$AAc?$AAh?$AA?$AA@ 10001c60     tchmdd:tchmain.obj
 0001:00000c90       ??_C@_1HK@OAECBAJK@?$AAC?$AA?3?$AA?2?$AAy?$AAm?$AAz?$AAk?$AAi?$AA?2?$AAp?$AAu?$AAb?$AAl?$AAi?$AAc?$AA?2?$AAC?$AAO?$AAM?$AAM?$AAO?$AAN?$AA?2?$AAo?$AAa?$AAk?$AA?2?$AAd?$AAr?$AAi?$AAv?$AAe@ 10001c90     tchmdd:tchmain.obj
 0001:00000d0c       ??_C@_1BM@IOLIHJIC@?$AAA?$AAc?$AAt?$AAi?$AAv?$AAi?$AAt?$AAy?$AAE?$AAv?$AAe?$AAn?$AAt?$AA?$AA@ 10001d0c     tchmdd:tchmain.obj
 0001:00000d28       ??_C@_1BG@JBGCDLHB@?$AAS?$AAy?$AAs?$AAt?$AAe?$AAm?$AA?2?$AAG?$AAW?$AAE?$AA?$AA@ 10001d28     tchmdd:tchmain.obj
 0001:00000d64       ?TouchDriverCalibrationPointGet@@YAHPAUTPDC_CALIBRATION_POINT@@@Z 10001d64 f   touch.obj
 0001:00000f74       DdsiTouchPanelAttach       10001f74 f   touch.obj
 0001:0000125c       DdsiTouchPanelDetach       1000225c f   touch.obj
 0001:0000133c       DdsiTouchPanelDisable      1000233c f   touch.obj
 0001:0000135c       DdsiTouchPanelEnable       1000235c f   touch.obj
 0001:00001390       DdsiTouchPanelGetDeviceCaps 10002390 f   touch.obj
 0001:0000153c       ?FilterSamples@@YAHPAUT_POSITION@@KK0@Z 1000253c f   touch.obj
 0001:00001854       DdsiTouchPanelGetPoint     10002854 f   touch.obj
 0001:00001bb0       DdsiTouchPanelPowerHandler 10002bb0 f   touch.obj
 0001:00001c14       DdsiTouchPanelSetMode      10002c14 f   touch.obj
 0001:00001d28       TouchPanelSetCalibration   10002d28 f   tch_cal:calibrat.obj
 0001:0000248c       ComputeMatrix33            1000348c f   tch_cal:calibrat.obj
 0001:00002658       TouchPanelCalibrateAPoint  10003658 f   tch_cal:calibrat.obj
 0001:00002794       ErrorAnalysis              10003794 f   tch_cal:calibrat.obj
 0001:00002a28       LargeNumSet                10003a28 f   tch_cal:largenum.obj
 0001:00002ae4       IsLargeNumNotZero          10003ae4 f   tch_cal:largenum.obj
 0001:00002b64       IsLargeNumNegative         10003b64 f   tch_cal:largenum.obj
 0001:00002bb0       IsLargeNumMagGreaterThan   10003bb0 f   tch_cal:largenum.obj
 0001:00002c9c       IsLargeNumMagLessThan      10003c9c f   tch_cal:largenum.obj
 0001:00002d88       LargeNumMagInc             10003d88 f   tch_cal:largenum.obj
 0001:00002e4c       LargeNumMagAdd             10003e4c f   tch_cal:largenum.obj
 0001:00002f9c       LargeNumMagSub             10003f9c f   tch_cal:largenum.obj
 0001:000030f0       LargeNumAdd                100040f0 f   tch_cal:largenum.obj
 0001:00003200       LargeNumSub                10004200 f   tch_cal:largenum.obj
 0001:00003310       LargeNumMulUint32          10004310 f   tch_cal:largenum.obj
 0001:00003478       LargeNumMulInt32           10004478 f   tch_cal:largenum.obj
 0001:00003554       LargeNumMult               10004554 f   tch_cal:largenum.obj
 0001:00003744       LargeNumSignedFormat       10004744 f   tch_cal:largenum.obj
 0001:00003834       LargeNumRAShift            10004834 f   tch_cal:largenum.obj
 0001:00003a90       LargeNumDivInt32           10004a90 f   tch_cal:largenum.obj
 0001:00003d60       LargeNumBits               10004d60 f   tch_cal:largenum.obj
 0001:00003e54       LargeNumToAscii            10004e54 f   tch_cal:largenum.obj
 0001:0000403c       TouchPanelDllEntry         1000503c f   tchmdd:tchbasic.obj
 0001:000041ac       DllMain                    100051ac f   tchmdd:tchbasic.obj
 0001:000041e8       TouchPanelGetDeviceCaps    100051e8 f   tchmdd:tchmain.obj
 0001:00004294       TouchPanelSetMode          10005294 f   tchmdd:tchmain.obj
 0001:0000436c       TouchPanelPowerHandler     1000536c f   tchmdd:tchmain.obj
 0001:00004388       TouchPanelEnable           10005388 f   tchmdd:tchmain.obj
 0001:00004fe8       TouchPanelDisable          10005fe8 f   tchmdd:tchmain.obj
 0001:000051bc       TouchPanelReadCalibrationPoint 100061bc f   tchmdd:tchmain.obj
 0001:00005410       TouchPanelReadCalibrationAbort 10006410 f   tchmdd:tchmain.obj
 0001:0000547c       SetEvent                   1000647c f i tchmdd:tchmain.obj
 0001:000054b4       SetLastError               100064b4 f   coredll:COREDLL.dll
 0001:000054c4       InterruptDone              100064c4 f   coredll:COREDLL.dll
 0001:000054d4       DeviceIoControl            100064d4 f   coredll:COREDLL.dll
 0001:000054e4       CreateFileW                100064e4 f   coredll:COREDLL.dll
 0001:000054f4       KernelIoControl            100064f4 f   coredll:COREDLL.dll
 0001:00005504       NKDbgPrintfW               10006504 f   coredll:COREDLL.dll
 0001:00005514       CloseHandle                10006514 f   coredll:COREDLL.dll
 0001:00005524       InterruptMask              10006524 f   coredll:COREDLL.dll
 0001:00005534       RegCloseKey                10006534 f   coredll:COREDLL.dll
 0001:00005544       RegQueryValueExW           10006544 f   coredll:COREDLL.dll
 0001:00005554       RegOpenKeyExW              10006554 f   coredll:COREDLL.dll
 0001:00005564       DisableThreadLibraryCalls  10006564 f   coredll:COREDLL.dll
 0001:00005574       RegisterDbgZones           10006574 f   coredll:COREDLL.dll
 0001:00005584       LeaveCriticalSection       10006584 f   coredll:COREDLL.dll
 0001:00005594       EnterCriticalSection       10006594 f   coredll:COREDLL.dll
 0001:000055a4       CeSetThreadPriority        100065a4 f   coredll:COREDLL.dll
 0001:000055b4       CreateThread               100065b4 f   coredll:COREDLL.dll
 0001:000055c4       InterruptInitialize        100065c4 f   coredll:COREDLL.dll
 0001:000055d4       InterruptDisable           100065d4 f   coredll:COREDLL.dll
 0001:000055e4       InitializeCriticalSection  100065e4 f   coredll:COREDLL.dll
 0001:000055f4       CreateEventW               100065f4 f   coredll:COREDLL.dll
 0001:00005604       ExitThread                 10006604 f   coredll:COREDLL.dll
 0001:00005614       GetTickCount               10006614 f   coredll:COREDLL.dll
 0001:00005624       WaitForSingleObject        10006624 f   coredll:COREDLL.dll
 0001:00005634       EventModify                10006634 f   coredll:COREDLL.dll
 0001:00005644       DeleteCriticalSection      10006644 f   coredll:COREDLL.dll
 0001:00005654       OpenEventW                 10006654 f   coredll:COREDLL.dll
 0001:00005664       __security_init_cookie     10006664 f   corelib0:seccinit.obj
 0001:0000572c       __GSHandlerCheck           1000672c f   corelib0:gshandler.obj
 0001:00005774       __GSHandlerCheckCommon     10006774 f   corelib0:gshandler.obj
 0001:0000581c       __security_check_cookie    1000681c f   corelib0:armsecgs.obj
 0001:00005830       __gsfailure                10006830 f   corelib0:armsecgs.obj
 0001:00005874       __rt_sdiv                  10006874 f   corelib1:COREDLL.dll
 0001:00005884       __rt_udiv                  10006884 f   corelib1:COREDLL.dll
 0001:00005894       memcpy                     10006894 f   corelib1:COREDLL.dll
 0001:000058a4       __security_gen_cookie2     100068a4 f   corelib1:COREDLL.dll
 0001:000058b4       __report_gsfailure         100068b4 f   corelib1:COREDLL.dll
 0001:000058dc       __IMPORT_DESCRIPTOR_COREDLL 100068dc     coredll:COREDLL.dll
 0001:000058f0       __NULL_IMPORT_DESCRIPTOR   100068f0     coredll:COREDLL.dll
 0002:00000000       __imp_SetLastError         10007000     coredll:COREDLL.dll
 0002:00000004       __imp_InterruptDone        10007004     coredll:COREDLL.dll
 0002:00000008       __imp_DeviceIoControl      10007008     coredll:COREDLL.dll
 0002:0000000c       __imp_CreateFileW          1000700c     coredll:COREDLL.dll
 0002:00000010       __imp_KernelIoControl      10007010     coredll:COREDLL.dll
 0002:00000014       __imp_NKDbgPrintfW         10007014     coredll:COREDLL.dll
 0002:00000018       __imp_CloseHandle          10007018     coredll:COREDLL.dll
 0002:0000001c       __imp_InterruptMask        1000701c     coredll:COREDLL.dll
 0002:00000020       __imp_RegCloseKey          10007020     coredll:COREDLL.dll
 0002:00000024       __imp_RegQueryValueExW     10007024     coredll:COREDLL.dll
 0002:00000028       __imp_RegOpenKeyExW        10007028     coredll:COREDLL.dll
 0002:0000002c       __imp_DisableThreadLibraryCalls 1000702c     coredll:COREDLL.dll
 0002:00000030       __imp_RegisterDbgZones     10007030     coredll:COREDLL.dll
 0002:00000034       __imp_LeaveCriticalSection 10007034     coredll:COREDLL.dll
 0002:00000038       __imp_EnterCriticalSection 10007038     coredll:COREDLL.dll
 0002:0000003c       __imp_CeSetThreadPriority  1000703c     coredll:COREDLL.dll
 0002:00000040       __imp_CreateThread         10007040     coredll:COREDLL.dll
 0002:00000044       __imp_InterruptInitialize  10007044     coredll:COREDLL.dll
 0002:00000048       __imp_InterruptDisable     10007048     coredll:COREDLL.dll
 0002:0000004c       __imp_InitializeCriticalSection 1000704c     coredll:COREDLL.dll
 0002:00000050       __imp_CreateEventW         10007050     coredll:COREDLL.dll
 0002:00000054       __imp_ExitThread           10007054     coredll:COREDLL.dll
 0002:00000058       __imp_GetTickCount         10007058     coredll:COREDLL.dll
 0002:0000005c       __imp_WaitForSingleObject  1000705c     coredll:COREDLL.dll
 0002:00000060       __imp_EventModify          10007060     coredll:COREDLL.dll
 0002:00000064       __imp_DeleteCriticalSection 10007064     coredll:COREDLL.dll
 0002:00000068       __imp_OpenEventW           10007068     coredll:COREDLL.dll
 0002:0000006c       __imp___rt_sdiv            1000706c     corelib1:COREDLL.dll
 0002:00000070       __imp___rt_udiv            10007070     corelib1:COREDLL.dll
 0002:00000074       __imp_memcpy               10007074     corelib1:COREDLL.dll
 0002:00000078       __imp___security_gen_cookie2 10007078     corelib1:COREDLL.dll
 0002:0000007c       __imp___report_gsfailure   1000707c     corelib1:COREDLL.dll
 0002:00000080       \177COREDLL_NULL_THUNK_DATA 10007080     coredll:COREDLL.dll
 0002:00000088       gIntrTouch                 10007088     touch.obj
 0002:00000150       dpCurSettings              10007150     tchmdd:tchmain.obj
 0002:00000594       gdwTouchIstTimeout         10007594     tchmdd:tchmain.obj
 0002:00000598       v_pfnSetCalibration        10007598     tchmdd:tchmain.obj
 0002:0000059c       v_pfnGetDeviceCaps         1000759c     tchmdd:tchmain.obj
 0002:000005a0       v_pfnSetMode               100075a0     tchmdd:tchmain.obj
 0002:000005a4       v_pfnPowerHandler          100075a4     tchmdd:tchmain.obj
 0002:000005a8       v_pfnEnableTest            100075a8     tchmdd:tchmain.obj
 0002:000005ac       v_pfnDisableTest           100075ac     tchmdd:tchmain.obj
 0002:000005b0       v_pfnReadCalibrationPointTest 100075b0     tchmdd:tchmain.obj
 0002:000005b4       v_pfnCalibrationPointAbortTest 100075b4     tchmdd:tchmain.obj
 0002:000005b8       __security_cookie          100075b8     corelib0:seccinit.obj
 0002:000005bc       __security_cookie_complement 100075bc     corelib0:seccinit.obj
 0002:000005c4       gIntrTouchChanged          100075c4     touch.obj
 0002:000006a4       v_pfnCgrCallback           100076a4     tchmdd:tchbasic.obj
 0002:000006d4       _bTchThreadHighPriority    100076d4     tchmdd:tchmain.obj
 0002:000006d8       hThread                    100076d8     tchmdd:tchmain.obj
 0002:000006e0       v_pfnPointCallback         100076e0     <common>
 0002:000006e4       CalibrationState           100076e4     <common>
 0002:000006e8       ghevCalibrationActivity    100076e8     <common>
 0002:000006ec       culReferenceCount          100076ec     <common>
 0002:000006f0       DisplayHeight              100076f0     <common>
 0002:00000700       csMutex                    10007700     <common>
 0002:00000714       hTouchPanelEvent           10007714     <common>
 0002:00000718       hCalibrationSampleAvailable 10007718     <common>
 0002:0000071c       DisplayWidth               1000771c     <common>
 0002:00000720       lCalibrationYCoord         10007720     <common>
 0002:00000724       lCalibrationXCoord         10007724     <common>
 0002:00000728       v_pfnCgrPointCallback      10007728     <common>

 entry point at        0001:0000403c

 Static symbols

 0001:00004660       TouchPanelpDetach          10005660 f   tchmdd:tchmain.obj
 0001:00004664       TouchPanelpAttach          10005664 f   tchmdd:tchmain.obj
 0001:00004768       TouchPanelpISR             10005768 f   tchmdd:tchmain.obj
 0001:00004dd4       TouchPanelpGetPriority     10005dd4 f   tchmdd:tchmain.obj
